:100000000EC026C025C05FC023C022C021C020C0B2
:100010001FC01EC01DC01CC01BC01AC019C01124A7
:100020001FBECFEDCDBF10E0A0E6B0E0E4EAF4E003
:1000300002C005900D92A836B107D9F710E0A8E6E6
:10004000B0E001C01D92A53BB107E1F702D028C284
:10005000D7CF8EEF88BB91E097BB2CE020BF89B74C
:10006000806489BF8FEA8EBD29BD93BF80E090E098
:100070000CD2813039F581E090E00FD29093A80046
:100080008093A7008091A7009091A800807790703E
:1000900024E0969587952A95E1F768E572E0D4D13A
:1000A0009093AA008093A9008091A9009091AA0042
:1000B000009731F480E797E19093AA008093A9001C
:1000C0007894FFCFFFCF1F920F920FB60F9211249B
:1000D000EF92FF922F933F934F935F936F937F9392
:1000E0008F939F93AF93BF93CF93DF93EF93FF9340
:1000F0001FBC8091AF009091B00001969093B0002A
:100100008093AF0080916A0090916B00009751F04E
:1001100080916A0090916B00019790936B0080939F
:100120006A007DC18091AB009091AC0001969093E4
:10013000AC008093AB002091AB003091AC00E0911B
:10014000A500F091A600EE59FF4F808190E028179E
:1001500039070CF464C11092AC001092AB0080918E
:10016000B100803A21F08091B100803859F48FEFCE
:100170009FEF9093AE008093AD0010926D001092AF
:100180006C0027C08091A3009091A400009731F0EB
:100190008091A3009091A400019717C08091AD00B9
:1001A0009091AE0001979093AE008093AD00809146
:1001B000AD009091AE00009761F480916C00909139
:1001C0006D00009731F482E090E09093A40080935A
:1001D000A3008091AD009091AE0097FF16C1809171
:1001E0006C0090916D00009709F0AEC080916000A6
:1001F000909161000196909361008093600020913E
:100200006000309161008091B20090E00197281762
:1002100039070CF472C010926900109268002091A6
:100220006800309169008091660090E028173907D6
:1002300011F1109266008091660090E0880F991F7E
:1002400003962BD1EC018093B3009093B4007E0110
:100250009F2D1BD1482F8093B200BE016F5F7F4F4F
:100260008EE690E050E002D11FBC88E59BE19093C0
:10027000B0008093AF002091AF003091B00080912A
:10028000A9009091AA0082179307A4F41092B000DD
:100290001092AF0080916E0090E090936100809387
:1002A000600010926100109260001092A6001092FF
:1002B000A50023C080916E0090E090936100809330
:1002C000600086B390E086709070959587959093C6
:1002D000A6008093A5008091A7009091A80080FFC0
:1002E0000CC08091A5009091A60080959095837098
:1002F00090709093A6008093A50087E090E0909383
:100300006D0080936C00E0916000F0916100E25913
:10031000FF4F81818093B10009C080916C00909162
:100320006D00019790936D0080936C008091B100F7
:1003300020916C0030916D0090E002C095958795FA
:100340002A95E2F780FDE9CF80916C0090916D00D5
:10035000019790936D0080936C008091B1008F3E67
:1003600029F41092AE001092AD004FC08091B10000
:10037000803A39F481E090E09093AE008093AD0034
:1003800008C08091B100803859F41092AE001092EC
:10039000AD0084E690E090936B0080936A0035C0D6
:1003A0008091B1008C3751F485B7877E806185BF1D
:1003B000F89485B7806285BF889527C04091B100C9
:1003C00080916C0090916D0021E030E0B90102C095
:1003D000660F771F8A95E2F7CB0150E084239523BF
:1003E0009093AE008093AD008091AD009091AE00EF
:1003F000009739F083E090E09093AE008093AD00D9
:1004000004C03093AE002093AD008091AD00909178
:10041000AE00009711F082E401C082E08ABDFF9136
:10042000EF91DF91CF91BF91AF919F918F917F918C
:100430006F915F914F913F912F91FF90EF900F90AF
:100440000FBE0F901F9018955527002480FF02C003
:10045000060E571F660F771F6115710521F09695DF
:100460008795009799F7952F802D0895A82F862FAF
:10047000E82FE199FECF1FBA05C0EEBBE09AE395E5
:100480000DB20D924150C8F70895E199FECF1FBA01
:100490008EBBE09A99278DB30895A8E142E0E8CF9A
:0404A000F894FFCFFE
:0804A400FF00011E642C63003F
:00000001FF
